:1000000011298030A100FE30AF200130AF207530C3
:10001000A7003030C628A101A117AF00AF08031D0B
:100020001328030114280130AF020310A20CA20C04
:10003000A20CC0302205403EAF07FE30AF202F0893
:10004000AF28A101A117AF00FE30AF202F08AF28C5
:10005000A401AA00AB01A01124080319A0150530C2
:10006000A3002730A900103041200330A900E83058
:100070004120A90164304120A9010A3041202A0809
:100080004828A8002B08A7002A08A600DA2026087E
:10009000A600A3030319A011240803195228230260
:1000A000031859282608031DA011A0195928303E0D
:1000B000AF280800A300240803190C292308AF2047
:1000C000A4035B28AD000611861183160611861164
:1000D0000F30860583122D08A0188C283E30A7000B
:1000E0008030C6203330AC00A0201330A700883009
:1000F000C620A0206430C520A0206430C520223056
:10010000AC00A02028308B200C308B2006308B20B8
:10011000A0142D088C282014AC00201C9A288611CD
:10012000033C031C9F289F200530A700DC30C6201D
:10013000031408002014FE3C0319AD288615201C6A
:10014000201006150F3086052C08F039860406119C
:10015000AC0E2018A0283230C5202D080C29A11B78
:10016000622883178001840AFF3E031DB2280C29F0
:10017000A901A800FF30A807031CA907031C0C292C
:100180000330A700DF30C620BA28A701E83EA6004A
:10019000A709FC30031CCF28A6070318CC28A60704
:1001A0000000A70FCC282618D528A61CD9280000A7
:1001B000D9280800AB01AA011030AC00270DAA0D08
:1001C000AB0D2808AA022908031C290FAB0203184B
:1001D000F0282808AA0729080318290FAB070310DD
:1001E000A60DA70DAC0BDE2826080C291030B00098
:1001F000A701A601AD0CAC0C031C04292808A60716
:1002000029080318290FA707A70CA60CAB0CAA0CEA
:10021000B00BFA282A080C29831383120313000059
:100220000800A00107309F00E03083168500FF30F2
:10023000860081138312850186012030840060309E
:10024000B220A03084005030B22020308400303002
:10025000B120C830B82001207730622062206220AF
:100260002E3062207030622069306220633062205C
:100270006230622061306220733062206930622017
:10028000633062202E3062206E3062206C3062203B
:100290000B30A900B830B92001204430622043302F
:1002A0006220463062203130622036306220553084
:1002B00062204B3062204430622020306220622075
:1002C000563062202D306220323062200730A90083
:1002D000D030B920012041306220643062206A3081
:1002E00062207530622073306220743062202030CA
:1002F00062204C30622044306220523062208618E6
:100300008729851F85290514862905107F29012045
:10031000533062206530622061306220723062208A
:1003200063306220683062202030622073306220A7
:1003300069306220673062206E3062206130622056
:100340006C306220361405128316051283123A2A85
:10035000C5013B03A500C90149082502031CC129A9
:10036000E421B61DBF294508A6004908A200A60140
:10037000A20A0314A60DA20BBA292608C504C90FA8
:10038000AC29B2014508B100B20CB10CB20CB10CF1
:10039000B20CB10CB20CB10C0F30B2053208AD008A
:1003A0003108AC00A9010A30A800F620B1002B08E2
:1003B000B200B4014508B3000F30B3050030B405F6
:1003C00031083307C5000800BA01B9010618F92938
:1003D0000130B820B90A0319BA0A0B303A02031CDB
:1003E000F829031DF729B9303902031CF829302DEB
:1003F000E6299B30B8200618B615061CB611361C27
:100400001A2A460EB100B200F030B1050F30B20525
:100410003208A7003108A600A9013A30A800DA2066
:10042000BC008030A1000230A2003C080D20FF304B
:1004300062202D2A8030A1000130A2003C080D204E
:100440000230A400460829200301B618013EB6195F
:10045000013A0319B610031DB614C60A85140130FB
:10046000A900F430B9208510A901F030A8002808AF
:10047000B9200800BE01C6013612361AD72ABA01C1
:10048000B901061C542AB90A0319BA0A0130B82066
:10049000AF303A02031C532A031D522AC9303902D5
:1004A000031C532A302D412ABA01B9010618902A9B
:1004B000B90A0319BA0A0A30B8203618842A39084A
:1004C0000B3A3A04031D6F2A8030A1000130A200CC
:1004D0003C080D203530622039306220832A3908EB
:1004E000193A3A04031D762A8514832A39084B3AAF
:1004F0003A04031D7D2A8510832A3908FA3A3A0402
:10050000031D832A302D8F2A11303A02031C8F2AB3
:10051000031D8E2A95303902031C8F2A302D562A4E
:1005200041303E02031C952A302DBE0A3A08031DB5
:100530009D2A65303902031C9E2A3616361CD62A9F
:100540003E0EB100B200F030B1050F30B2053208F6
:10055000A7003108A600A9014130A800DA20BC009C
:100560008030A10080302120463062206F30622030
:10057000753062206E30622064306220203062204C
:100580007330622069306220673062206E306220F2
:10059000613062206C306220203062208030A10007
:1005A0000230A2003C080D20FF3062203D2A361C9C
:1005B000FB2A0120493062206E30622069306220BF
:1005C0007430622069306220613062206C306220B9
:1005D000693062207A306220653062202E306220DD
:1005E000622062208030A100C03021201030A400A1
:1005F0005F305A206A2B0730BC000130A2003C0853
:100600000B20A101361D132B3B30420203180A2B8D
:10061000C20A122BC20117303F020318112BBF0A66
:10062000122BBF01172B4308C2004008BF00051B57
:10063000272B3F08031D1F2B0C30C100262B0D302C
:100640003F02031C262B0C303F02C1002C2B3F081D
:10065000C1002030622062200A3041020318322B90
:10066000203062208030A100410828203A306220EA
:100670000230A400420829203A3062203030622043
:100680006220051B532B0C303F0203184C2B6130AA
:1006900062206D306220502B703062206D306220FD
:1006A0000D30BC00552B0F30BC004208031901303F
:1006B000031D0301B5001E30420203190130031D62
:1006C00003013504B5000130861803013504031910
:1006D0006A2B082D361E062DE4210130C9000F308B
:1006E00049020318762BE421C90F6F2BB61036117F
:1006F000E421E421E421B61D7F2B0514802B051095
:100700001230C900143049020318892BE421C90FA3
:10071000822BE4210730BB00A8214508C300E42157
:10072000B61C932B36150630BB00A8214508C00027
:10073000E421B61C9C2B36150630BB00A8214508C9
:10074000BD000330BB00A8214508C7000530BB0031
:10075000A8214508C4000830BB00A8214508C800EE
:10076000E421B61CB42B3615361CBA2B3619B92B1E
:10077000361001203619052D8030A100C03021200F
:100780001030A40020305A2080302120A1010130F7
:100790004702031DD22B4D3062206F3062206E3035
:1007A0006220132C02304702031DDD2B54306220DF
:1007B0007530622065306220132C03304702031D20
:1007C000E82B573062206530622064306220132CA1
:1007D00004304702031DF32B54306220683062203E
:1007E00075306220132C05304702031DFE2B463066
:1007F00062207230622079306220132C063047026A
:10080000031D092C53306220613062207430622055
:10081000132C07304702031D132C53306220753010
:1008200062206E3062208030A100C03021203D085F
:1008300028202030622001304402031D2E2C4A3033
:100840006220613062206E3062207530622061303B
:1008500062207230622079306220EA2C0230440239
:10086000031D432C463062206530622062306220D6
:1008700072306220753062206130622072306220F6
:1008800079306220EA2C03304402031D522C4D3093
:1008900062206130622072306220633062206830F2
:1008A0006220EA2C04304402031D612C4130622096
:1008B0007030622072306220693062206C306220B9
:1008C000EA2C05304402031D6C2C4D30622061304F
:1008D000622079306220EA2C06304402031D792C14
:1008E0004A306220753062206E30622065306220AE
:1008F000EA2C07304402031D862C4A3062207530F2
:1009000062206C30622079306220EA2C0830440288
:10091000031D972C413062207530622067306220C1
:10092000753062207330622074306220EA2C093006
:100930004402031DAE2C53306220653062207030BB
:10094000622074306220653062206D306220623037
:1009500062206530622072306220EA2C0A30440244
:10096000031DC12C4F30622063306220743062203E
:100970006F30622062306220653062207230622007
:10098000EA2C0B304402031DD62C4E3062206F300F
:10099000622076306220653062206D3062206230E5
:1009A00062206530622072306220EA2C0C304402F2
:1009B000031DEA2C443062206530622063306220DF
:1009C000653062206D3062206230622065306220C6
:1009D0007230622009304402031DF92C203062205D
:1009E000273062208030A1000230A400480829206E
:1009F000052D20306220323062203030622080307D
:100A0000A1000230A40048082920072D302D3A2AE1
:100A1000851F0F2D0512831605128312112D8316C3
:100A2000051683129B30B820420803190130031DBC
:100A30000301B50001308618030135040319212D87
:100A40000515851585140130A900F430B92005116C
:100A5000851185100130A9004A30B920C60A6D2BD6
:100A600001204E3062206F306220203062207330CF
:100A7000622069306220673062206E30622061300F
:100A800062206C306220203084006030B220A030C0
:100A900084005030B220203084003030B12006185D
:100AA000B616061CB61203010618013EB61A013C22
:100AB000031D602DB70A0319B80A0130B820532D61
:100AC0000301B61A0130013A0319B612031DB61616
:100AD00003010618013EB61A013C031D752DB70A25
:100AE0000319B80A0130B820682D03303802DE300F
:0C0AF000031937020318432D36143A2A6C
:02400E00503F21
:00000001FF
